:100000000C9463000C948B000C948B000C948B006C
:100010000C948B000C948B000C948B000C941B089C
:100020000C948B000C948B000C948B000C948B0024
:100030000C948B000C948B000C948B000C948B0014
:100040000C94D1070C948B000C949F070C947907A7
:100050000C948B000C948B000C948B000C948B00F4
:100060000C948B000C948B000000000023002600F1
:10007000290000000000240027002A0000000000E2
:10008000250028002B0004040404040404040202D4
:100090000202020203030303030301020408102007
:1000A0004080010204081020010204081020000012
:1000B0000008000201000003040700000000000027
:1000C0000000DB08D61111241FBECFEFD8E0DEBF41
:1000D000CDBF23E0A8E6B1E001C01D92A634B2076F
:1000E000E1F711E0A0E0B1E0ECE2F2E302C005903C
:1000F0000D92A836B107D9F710E0C2E6D0E004C0EF
:100100002197FE010E940A14C136D107C9F70E9447
:10011000A9090C9409190C9400000895AF92BF929C
:10012000CF92DF92EF92FF920F931F93CF93DF93C3
:100130006C017B018B01040F151FEB015E01AE18F2
:10014000BF08C017D10759F06991D601ED91FC9114
:100150000190F081E02DC6010995892B79F7C50141
:10016000DF91CF911F910F91FF90EF90DF90CF9093
:10017000BF90AF900895FC01538D448D252F30E042
:10018000842F90E0821B930B541710F0CF960895A4
:1001900001970895FC01918D828D981761F0A28DD1
:1001A000AE0FBF2FB11D5D968C91928D9F5F9F7397
:1001B000928F90E008958FEF9FEF0895FC01918D4D
:1001C000828D981731F0828DE80FF11D858D90E0BA
:1001D00008958FEF9FEF0895FC01918D228D892F57
:1001E00090E0805C9F4F821B91098F73992708953F
:1001F0008DEA91E00E94EC0021E0892B09F420E0D7
:10020000822F0895FC01A48DA80FB92FB11DA35A08
:10021000BF4F2C91848D90E001968F739927848F26
:10022000A689B7892C93A089B1898C918370806449
:100230008C93938D848D981306C00288F389E02DEA
:1002400080818F7D80830895EF92FF920F931F939B
:10025000CF93DF93EC0181E0888F9B8D8C8D981379
:100260001AC0E889F989808185FF15C09FB7F89485
:10027000EE89FF896083E889F989808183708064D1
:1002800080839FBF81E090E0DF91CF911F910F911C
:10029000FF90EF900895F62E0B8D10E00F5F1F4F2B
:1002A0000F731127E02E8C8D8E110CC00FB607FC3A
:1002B000FACFE889F989808185FFF5CFCE010E94C8
:1002C0000201F1CFEB8DEC0FFD2FF11DE35AFF4F33
:1002D000F0829FB7F8940B8FEA89FB898081806256
:1002E000CFCFCF93DF93EC01888D8823B9F0AA8913
:1002F000BB89E889F9898C9185FD03C0808186FDE1
:100300000DC00FB607FCF7CF8C9185FFF2CF80812F
:1003100085FFEDCFCE010E940201E9CFDF91CF91A1
:100320000895833081F028F4813099F08230A9F06B
:1003300008958730A9F08830C9F08430B1F48091F5
:1003400080008F7D03C0809180008F778093800034
:10035000089584B58F7784BD089584B58F7DFBCFD4
:100360008091B0008F778093B00008958091B000A5
:100370008F7DF9CF1F93CF93DF93282F30E0F901C2
:10038000E255FF4F8491F901E656FF4FD491F901F0
:10039000EA57FF4FC491CC23A9F0162F81110E9478
:1003A0009101EC2FF0E0EE0FFF1FE458FF4FA591F5
:1003B000B4918FB7F894EC91111108C0D095DE2359
:1003C000DC938FBFDF91CF911F910895DE2BF8CF83
:1003D000CF93DF93EC01809130039091310302972A
:1003E00049F4C130D10509F43BC06CF560E02097B9
:1003F00009F437C08091300390913103049749F498
:10040000C130D10509F45CC00CF037C0209709F465
:1004100042C08091300390913103059709F0E5C007
:10042000CA30D10508F0E1C0FE01E75EFD4F0C9433
:100430000A14780284029502AB02C602C802CF02F7
:10044000DB02EC02F302C230D105A9F060E0C33058
:10045000D10581F6809134030E94BA0160E006C0A4
:1004600061E0809134030E94BA0161E0809136031B
:100470000E94BA01BFCF61E0EDCFC230D10539F1A2
:10048000C330D10509F0C5CF61E0809134030E94EB
:10049000BA0160E022C061E0809134030E94BA0199
:1004A00060E0809136030E94BA0161E080913803D8
:1004B0000E94BA0160E080913A030E94BA01A9CF7C
:1004C00060E0809134030E94BA0161E0EACF60E00D
:1004D000809134030E94BA0161E0809136030E944A
:1004E000BA0160E0809138030E94BA0161E0E3CF75
:1004F00060E0809134030E94BA0161E0809136038C
:100500000E94BA0161E00BC060E0809134030E9458
:10051000BA0161E0809136030E94BA0160E08091E7
:1005200038030E94BA0160E010C060E0809134039B
:100530000E94BA0161E0809136030E94BA0160E036
:10054000809138030E94BA0161E080913A030E94D1
:10055000BA0161E015C060E0809134030E94BA01E5
:1005600061E0809136030E94BA0160E08091380317
:100570000E94BA0161E080913A030E94BA0160E0F2
:1005800080913C03DF91CF910C94BA0161E0E4CFFC
:1005900061E0809134030E94BA0160E0E2CF61E043
:1005A000809134030E94BA0160E0809136030E947A
:1005B000BA0161E0DBCF61E0809134030E94BA01AF
:1005C00060E0809136030E94BA0161E080913803B7
:1005D0000E94BA0160E0CFCF61E0809134030E94B5
:1005E000BA0160E08BCF60E0F8CFDF91CF91089542
:1005F000CF93DF9390E0FC01E656FF4F24918A579A
:100600009F4FFC0184918823D1F090E0880F991FBF
:10061000FC01EE58FF4FA591B491FC01E458FF4F47
:10062000C591D49161110EC09FB7F8948C91E22FBF
:10063000E0958E238C932881E223E8839FBFDF918E
:10064000CF9108958FB7F894EC91E22BEC938FBF84
:10065000F6CFCF93DF93EC0161E085E00E94F802D2
:10066000209731F460E085E0DF91CF910C94BA01DE
:10067000CF3FD10511F461E0F6CFE3EBF0E0E49178
:10068000E33029F140F4E130B1F0E230D9F0C03884
:10069000D1058CF7E7CFE73021F1E83051F1E430B4
:1006A000B1F780918000806280938000D0938B00AE
:1006B000C0938A0004C084B5806884BDC7BDDF9143
:1006C000CF91089584B5806284BDC8BDF8CF809174
:1006D0008000806880938000D0938900C093880058
:1006E000EECF8091B00080688093B000C093B300DB
:1006F000E6CF8091B00080628093B000C093B400D8
:10070000DECF3FB7F89480916D0190916E01A0917A
:100710006F01B091700126B5A89B05C02F3F19F05D
:100720000196A11DB11D3FBFBA2FA92F982F882771
:10073000BC01CD01620F711D811D911D42E0660F4C
:10074000771F881F991F4A95D1F708954F925F929E
:100750006F927F928F929F92AF92BF92EF92FF9291
:100760000F931F93CF93DF93EC0197FF04C0CC2727
:10077000DD27C81BD90B181619060CF061C081E0E3
:1007800090E0909329038093280304E010E08AE02E
:10079000E82EF12C209709F46FC00E94810380900D
:1007A0003E0390903F03A0904003B09041032B0183
:1007B0003C01481859086A087B0880902A039090E9
:1007C0002B03A0902C03B0902D03481459046A0405
:1007D0007B0400F360933E0370933F0380934003D8
:1007E0009093410380913203909133032091280329
:1007F000309129032130310559F501969093330347
:100800008093320320912E0330912F038217930798
:1008100021F4109233031092320321978091320316
:10082000909133032091300330913103B70125308B
:10083000310509F0B8010E94D7130E94E801AACF40
:10084000892B09F4A2CF10922903109228039DCF7F
:10085000892B41F480912E0390912F0390933303C1
:1008600080933203809132039091330301979093E8
:10087000330380933203D1CFDF91CF911F910F913A
:10088000FF90EF90BF90AF909F908F907F906F9070
:100890005F904F9008958F929F92AF92BF92CF92A8
:1008A000DF92EF92FF926B017C010E9481034B016A
:1008B0005C01C114D104E104F104B9F00E94810388
:1008C000681979098A099B09683E73408105910579
:1008D00080F321E0C21AD108E108F10888EE880E01
:1008E00083E0981EA11CB11CE4CFFF90EF90DF9035
:1008F000CF90BF90AF909F908F900895CF92DF924E
:10090000EF92FF920F931F93CF93DF93442331F124
:100910008C01D0E0C0E06B01770FEE08FF0861E0CA
:1009200081E10E94BA01C701B6010E944B0460E058
:1009300081E10E94BA0162E370E080E090E00E94F1
:100940004B0421960C171D0751F7DF91CF911F9192
:100950000F91FF90EF90DF90CF9008956E5C7F4FE6
:10096000072E000C880B990BDF91CF911F910F91EF
:10097000FF90EF90DF90CF900C944B0460E086E006
:100980000E94BA0160E087E00E94BA0160E088E05E
:100990000E94BA0160E089E00C94BA01EF92FF92E4
:1009A0000F931F93CF93DF937C010DE811E0D0E00C
:1009B000C0E0F80161918F01C7018C0F9D1F0E945B
:1009C00068132196C032D105A1F780E290E0DF9153
:1009D000CF911F910F91FF90EF9008958091760134
:1009E000909177010C94CE04CF93DF93EC0181E0DA
:1009F00090E09093A4018093A30110929201109231
:100A000091010E94EE04CE010E94A6038091A501EF
:100A10009091A601009739F482E090E090939201C2
:100A20008093910103C081309105C1F31092A4011C
:100A30001092A30182E090E09093A6018093A5011B
:100A40000E94EE04DF91CF910C94BE040F931F938C
:100A5000CF93DF93CDE8D1E08C010D581140C80150
:100A60008C0F9D1F0E946013899381E0CD3AD807B7
:100A7000B1F780E290E0DF91CF911F910F9108953F
:100A8000FC0180819181009711F00C94001260E0CC
:100A900070E0CB0108950F931F93CF93DF938C01E8
:100AA000EB01FC01808191810097E1F068817981FF
:100AB00061157105A9F0428153812C813D81421756
:100AC000530770F00E9431168C819D81F801958347
:100AD00084831D821C82DF91CF911F910F91089515
:100AE0000E94E21488819981F801918380838A8130
:100AF0009B81938382838C819D81958384831982DA
:100B000018821B821A82E5CFCF93DF93EC01888194
:100B10009981009711F00E94E214198218821D82B7
:100B20001C821B821A82DF91CF910895FC01808183
:100B30009181009711F00C94E21408950F931F9384
:100B4000CF93DF93EC0188819981009759F02A8136
:100B50003B812617370730F081E0DF91CF911F915D
:100B60000F9108958B016F5F7F4F0E946B15009767
:100B700059F0998388831B830A832C813D81232B21
:100B800059F7FC011082E8CF80E0E7CFEF92FF92A7
:100B90000F931F93CF93DF93EC01FB01E080F18073
:100BA000E114F10411F10481158101151105A9F079
:100BB0008C819D81080F191FB801CE010E949E05EE
:100BC000882399F0288139818C819D81B701820F1A
:100BD000931F0E9431161D830C83CE01DF91CF91AC
:100BE0001F910F91FF90EF900895CE010E94840510
:100BF000F4CFEF92FF920F931F93CF93DF93EC010B
:100C00007B018A01BA010E949E0581110BC0CE01B1
:100C10000E948405CE01DF91CF911F910F91FF902B
:100C2000EF9008951D830C83B701888199810E94FC
:100C30003116F0CFFC0111821082138212821582CC
:100C4000148250E040E06BE371E00C94F905FB0185
:100C500001900020E9F73197AF01461B570B0C9428
:100C6000F905CF93DF9300D0CDB7DEB7FC01118239
:100C70001082138212821582148269831A82BE0145
:100C80006F5F7F4F0E9427060F900F90DF91CF91EB
:100C90000895CF93DF93EC01FB018617970749F086
:100CA000608171816115710541F0448155810E9417
:100CB000F905CE01DF91CF9108950E948405F9CF07
:100CC000FF920F931F93CF93DF9300D0CDB7DEB782
:100CD00086E0F82E8DEA91E00E94EC00892B09F461
:100CE00076C08DEA91E00E94CA00833251F08E33C3
:100CF00009F049C06BE371E082E293E00E942706AD
:100D0000E9CF20911C0330911D0380912003909125
:100D1000210328173907F4F640911E0350911F0351
:100D200020911A0330911B03C901019690931B0374
:100D300080931A03F29EC001F39E900D112462E28B
:100D400073E0840F951F0E94490680911C039091C7
:100D50001D03019690931D0380931C0380911A0339
:100D600090911B032091200330912103281739070C
:100D70000CF0B0CF2F5F3F4F821B930B90931B0360
:100D800080931A03A7CF89831A82009126031091BA
:100D900027030F5F1F4FB80182E293E00E949E0578
:100DA000882309F497CF2091220330912303809167
:100DB000260390912703BE016F5F7F4F820F931F21
:100DC0000E943116109327030093260383CF0F90C0
:100DD0000F90DF91CF911F910F91FF9008950E9486
:100DE000F80081110C94600608950F931F93CF9320
:100DF000DF93CDB7DEB7A0970FB6F894DEBF0FBE76
:100E0000CDBF1F9293E29F937F936F93282F082E5D
:100E1000000C330B3F938F938CE291E09F938F9361
:100E20001F9280E28F938E010F5F1F4F1F930F93CE
:100E30000E943816F80101900020E9F73197AF01C0
:100E4000401B510BB8018DEA91E00E948E000FB655
:100E5000F894DEBF0FBECDBFA0960FB6F894DEBFEC
:100E60000FBECDBFDF91CF911F910F9108950F93CA
:100E70001F93CF93DF93CDB7DEB7A0970FB6F8944B
:100E8000DEBF0FBECDBF1F9293E29F937F936F9300
:100E9000282F082E000C330B3F938F9384E391E0AF
:100EA0009F938F931F9280E28F938E010F5F1F4F4E
:100EB0001F930F930E943816F80101900020E9F764
:100EC0003197AF01401B510BB8018DEA91E00E94B0
:100ED0008E000FB6F894DEBF0FBECDBFA0960FB642
:100EE000F894DEBF0FBECDBFDF91CF911F910F9160
:100EF00008951F920F920FB60F9211242F933F93D4
:100F00004F935F936F937F938F939F93AF93BF9311
:100F1000EF93FF938DEA91E00E940201FF91EF9120
:100F2000BF91AF919F918F917F916F915F914F9101
:100F30003F912F910F900FBE0F901F9018951F9209
:100F40000F920FB60F9211242F938F939F93EF93CD
:100F5000FF93E091BD01F091BE018081E091C3015A
:100F6000F091C40182FD1BC090818091C6018F5F0A
:100F70008F732091C701821741F0E091C601F0E024
:100F8000E355FE4F958F8093C601FF91EF919F919E
:100F90008F912F910F900FBE0F901F901895808109
:100FA000F4CF1F920F920FB60F9211242F933F93FD
:100FB0008F939F93AF93BF938091690190916A0142
:100FC000A0916B01B0916C013091680123E0230F77
:100FD0002D3758F50196A11DB11D2093680180930E
:100FE000690190936A01A0936B01B0936C018091A9
:100FF0006D0190916E01A0916F01B0917001019609
:10100000A11DB11D80936D0190936E01A0936F019E
:10101000B0937001BF91AF919F918F913F912F91AC
:101020000F900FBE0F901F90189526E8230F029681
:10103000A11DB11DD2CF1F920F920FB60F92112496
:101040002F933F934F935F936F937F938F939F93D0
:10105000AF93BF93CF93DF93EF93FF9320914A0217
:1010600030E0F901E255FF4F8491F901E656FF4F58
:10107000D491F901EA57FF4FC491CC2379F0811143
:101080000E949101EC2FF0E0EE0FFF1FE859FF4F97
:10109000A591B491EC91ED2381E009F480E02091D9
:1010A0004D0230914E022F5F3F4F30934E022093FE
:1010B0004D0290911703943618F095E090934B02EF
:1010C00090914B02933009F44CC0E0F4923011F14E
:1010D00090914C02992319F081116BC02D9AFF91C8
:1010E000EF91DF91CF91BF91AF919F918F917F91C0
:1010F0006F915F914F913F912F910F900FBE0F9085
:101100001F901895943009F448C0953009F7811163
:10111000DFCF09C08111DCCF20914D0230914E020A
:101120002436310528F410924E0210924D02D0CF91
:1011300010921703E091170391E09E0F909317030D
:10114000F0E020914D0230914E02EE0FFF1FE65B62
:10115000FD4F3683258310924E0210924D0293E08C
:1011600019C0813009F0B4CFE091170391E09E0FD0
:1011700090931703F0E020914D0230914E02EE0F54
:10118000FF1FE65BFD4F3683258310924E021092BF
:101190004D0294E090934B029BCF882359F220910B
:1011A0004D0230914E022536310508F491CF95E07D
:1011B000F1CF2D9894CFEF92FF920F931F93CF937F
:1011C000DF931092B0011092AF0188EE93E0A0E09F
:1011D000B0E08093B1019093B201A093B301B093BA
:1011E000B4018EE191E09093AE018093AD0185EC66
:1011F00090E09093BA018093B90184EC90E09093D1
:10120000BC018093BB0180EC90E09093BE01809381
:10121000BD0181EC90E09093C0018093BF0182EC0E
:1012200090E09093C2018093C10186EC90E090938E
:10123000C4018093C3011092C6011092C70110929D
:10124000C8011092C9011092330310923203109218
:1012500029031092280310923E0310923F0310922C
:1012600040031092410380E390E090932F0380931A
:101270002E0386E090E0909335038093340387E05B
:1012800090E0909337038093360388E090E090934A
:1012900039038093380389E090E090933B03809377
:1012A0003A0361E086E00E94F80261E08091360333
:1012B0000E94F80261E0809138030E94F80261E028
:1012C00080913A030E94F80210923D0310923C0371
:1012D00084E090E0909331038093300380934A023E
:1012E00010924C0282E293E00E941A0610921903B7
:1012F0001092180310921B0310921A0310921D03F0
:1013000010921C0384E190E09093210380932003CA
:1013100080E890E00E944614EC0125E130E029933A
:1013200039938E017C0120E8E20EF11CC8010E9475
:101330001A060A5F1F4FE016F106C1F7D0931F038C
:10134000C0931E03DF91CF911F910F91FF90EF90FB
:101350000895CF93DF93CDB7DEB7C555D1090FB64A
:10136000F894DEBF0FBECDBF789484B5826084BD93
:1013700084B5816084BD85B5826085BD85B5816099
:1013800085BD80916E00816080936E001092810017
:1013900080918100826080938100809181008160D2
:1013A0008093810080918000816080938000809193
:1013B000B10084608093B1008091B000816080931F
:1013C000B00080917A00846080937A0080917A00E6
:1013D000826080937A0080917A00816080937A00A5
:1013E00080917A00806880937A001092C100E09129
:1013F000BD01F091BE0182E08083E091B901F091DE
:10140000BA011082E091BB01F091BC018FEC8083A6
:101410001092C501E091C101F091C20186E0808384
:10142000E091BF01F091C001808180618083E091F3
:10143000BF01F091C001808188608083E091BF018D
:10144000F091C001808180688083E091BF01F091BC
:10145000C00180818F7D80838DEA91E00E94EC0045
:10146000892B29F08DEA91E00E94CA00F5CF61E056
:1014700081E10E94F80261E085E00E94F80261E0EB
:1014800082E00E94F80220912E0330912F03032E58
:10149000000C440B550B60E077E883E993E00E9471
:1014A000EB13CA01B9012AEE31E040E050E00E949E
:1014B000EB1320932A0330932B0340932C03509378
:1014C0002D030E94BE046BE371E082E293E00E9470
:1014D000270610927701109276011092750180E232
:1014E00090E09093740180937301909372018093C4
:1014F000710110E000E0FF24F394C8010E9426056A
:1015000080918D0190918E018336910531F4109375
:10151000770100937601F0927501005E1F4F01156F
:1015200024E0120751F70091760110917701809124
:101530007501882309F413C1C8010E942605109281
:101540008E0110928D01C8010E94CE04209173017A
:10155000309174018091760190917701820F931FF1
:10156000909377018093760160917101709172017F
:10157000269FA001279F500D369F500D11248417E0
:10158000950724F0109277011092760183E690E09F
:1015900090938E0180938D018091760190917701D7
:1015A0000E94CE0480919701882321F061E082E0BF
:1015B0000E94BA0164E670E080E090E00E944B0473
:1015C0008091930190919401019709F01BC1809142
:1015D0009501909196010E942903F89482E08093EE
:1015E000B0008093B10094E69093B3001092B200E3
:1015F00080937000789480934B021092170380912F
:101600004A0260E00E94F8024091A20166E970E09F
:1016100081E090E00E947E048E010F5F1F4F809159
:101620001C0390911D03181619060CF054C1CE012D
:10163000845B9F4F0E941A06CE018A5B9F4F0E94D7
:101640001A0680911C0390911D03009709F439C17B
:101650000CF0DBC0CE018E960E941A06BE01625DC0
:101660007F4FCE01845B9F4F0E944B05CE018E962B
:101670000E9496056296CEACDFAC6297AA24A39432
:10168000B12CC114D10421F05601CC24C394D12C27
:10169000C8010E941A066296EEACFFAC6297CE14A7
:1016A000DF0408F5AE14BF0408F475012E96EEAD04
:1016B000FFAD2E97EE0DFF1DB08010822E966EAD01
:1016C0007FAD2E976C0D7D1DC8016115710509F464
:1016D000E6C00E9427062E968EAD9FAD2E97E80E8F
:1016E000F91ED701BC92B801CE018A5B9F4F0E94C0
:1016F0004B05C8010E94960562968EAD9FAD62971C
:10170000892B09F4DEC02E96EEADFFAD2E973097F3
:1017100009F4D7C0E081E154E93108F0D2C00E2EBF
:10172000000CFF0BEA56F44F0C940A141A0EA90D84
:10173000540D990D6B0E2B0E610C520C610CE40DC7
:10174000610C830D780F610C2A0D610C610C610C2A
:10175000F50DA00E610C1C0D610CB00E650F83E63B
:1017600090E090938E0180938D01909390018093EF
:101770008F0181E090E0909392018093910110920B
:10178000940110929301109296011092950121E01C
:101790002093970182E090E09093990180939801C3
:1017A00042E150E050939B0140939A0140E450E0A5
:1017B00050939D0140939C0140E850E050939F015D
:1017C00040939E014EEF50E05093A1014093A00141
:1017D0002093A2011092A4011092A3019093A6015C
:1017E0008093A5011092A8011092A70188EB9BE0BD
:1017F0009093AA018093A9011092AC011092AB01C1
:10180000C801CECE90E080E0E6CE20911803309162
:10181000190346E0429FC001439F900D112460913F
:101820001E0370911F03680F791F1A8219821C8290
:101830001B821E821D82C8010E94490680911803E6
:1018400090911903019690931903809318032091A6
:101850001C0330911D032150310930931D03209347
:101860001C0320912003309121032817390744F4E9
:101870002F5F3F4F821B930B9093190380931803A4
:101880001FA61EA619AA18AA1BAA1AAAB801CE0139
:101890008E960E944B05C8010E949605DFCE0E94DD
:1018A000840519CF6AE071E0C8010E94311664E630
:1018B00070E080E090E00E944B04B80188E40E9450
:1018C000F506CE018A5B9F4F0E949605CE01845B90
:1018D0009F4F0E9496058FE492E090938A01809337
:1018E000890120901703312C30928C0120928B01BA
:1018F00080914B02853009F097C080915102909100
:101900005202885891098D35910508F06FC3809176
:101910001703843009F03CC3809153029091540224
:101920008097479708F034C38091550290915602F2
:101930000997099708F02CC310928801109287012B
:101940008FEF9FEFDC018093830190938401A0933C
:101950008501B093860181E090E0909380018093AF
:101960007F018091830190918401A0918501B091C4
:1019700086018F3FEFEF9E07AE07BE0709F0E5C374
:1019800080917B0190917C01A0917D01B0917E01BD
:101990008093830190938401A0938501B093860185
:1019A00080917B0190917C01A0917D01B0917E019D
:1019B0008736E8E99E07EAE9AE07E6EABE0709F4DA
:1019C000C5C40CF0E9C38D3F22E092072AE9A207C3
:1019D00026EAB20709F422C48D3D9242AA49B64ACA
:1019E00009F448C480919301909194010197B9F44E
:1019F00080919501909196018F3F910511F001978B
:101A000071F464E670E080E090E00E944B04409145
:101A1000A20164E670E082E090E00E947E0482E031
:101A200080934B02109217030E94F800882309F458
:101A3000F6CD0E946006F0CD66E071E0C8010E941C
:101A4000311664E670E080E090E00E944B04B8013B
:101A500086E535CF4091A20168EC70E081E090E02E
:101A60000E947E048091910190919201029751F021
:101A70001092A6011092A5018091A9019091AA014E
:101A80000E94F4044091A20164E670E082E090E0DC
:101A90000E947E046AE070E080E090E00E944B04C7
:101AA0006CE371E08FE40BCF4091A20168EC70E031
:101AB00081E090E00E947E048091910190919201DA
:101AC000019779F081E090E09093A6018093A501C1
:101AD0008091A9019091AA019195819591090E9407
:101AE000F4044091A20164E670E082E090E00E947C
:101AF0007E046AE070E080E090E00E944B0463E4C2
:101B000071E083E4DCCE81E090E0909394018093D7
:101B100093010E94EE0480919501909196010E949C
:101B2000290360919501709196018CE40E9437071A
:101B3000C8CE10929401109293010E94EE0490E09E
:101B400080E00E94290360918F017091900184E4EC
:101B5000EDCFCE018A5B9F4F0E94400597FD2EC0BE
:101B60006F3F71058105910509F05CF57093960151
:101B7000609395018091930190919401019719F4DC
:101B8000CB010E9429030E94EE04809196018F935D
:101B9000809195018F9385E691E09F938F931F939A
:101BA0000F930E946816B80182E40E94F5060F9018
:101BB0000F900F900F900F900F9083CE70E060E029
:101BC000D5CF6FEF70E0D2CF809196018F93809147
:101BD00095018F9385E691E09F938F931F930F93C9
:101BE0000E946816B8018AE4E0CF809192018F9339
:101BF000809191018F93809194018F9380919301B3
:101C00008F938091A4018F938091A3018F938091F2
:101C100090018F9380918F018F938AE491E09F933D
:101C20008F931F930F930E946816B80183E50E945B
:101C3000F5064BC08091AC018F938091AB018F93DF
:101C400083E591E09F938F931F930F930E946816F3
:101C5000B80181E4AACF1092A8011092A7011092B6
:101C6000A4011092A30182E090E09093A6018093DA
:101C7000A50181E090E090939201809391011092F0
:101C8000AC011092AB010E94EE048091AA018F93E7
:101C90008091A9018F938091A8018F938091A701D2
:101CA0008F938FE591E09F938F931F930F930E94E3
:101CB0006816B80186E40E94F5064091A20164E628
:101CC00070E082E090E00E947E040FB6F894DEBFE0
:101CD0000FBECDBFF6CD8091A7019091A801909342
:101CE000AA018093A9011092A4011092A30182E09D
:101CF00090E09093A6018093A50190939201809328
:101D0000910181E090E09093AC018093AB010E943F
:101D1000EE048091AA018F938091A9018F93809105
:101D2000A8018F938091A7018F938FE591E09F93F6
:101D30008F931F930F930E946816B80185E4BBCF61
:101D4000CE018A5B9F4F0E944005672B29F41092B9
:101D5000A2010E94EE04B5CD81E08093A201F9CFEB
:101D600048E9C42E41E0D42E52E0E52EF12C2C9609
:101D70008EAD9FAD2C97E816F90638F42896EEAD97
:101D8000FFAD2897309709F091C010927801E8E7ED
:101D9000F1E06081C8010E943106C70101972C96CD
:101DA0002EAD3FAD2C978217930738F42896EEADF1
:101DB000FFAD2897309709F07CC010927801E8E7D2
:101DC000F1E06081CE018E960E943106C701029734
:101DD0002C962EAD3FAD2C978217930738F428969A
:101DE000EEADFFAD2897309709F066C010927801EC
:101DF000E8E7F1E06081CE01CA960E9431061DAA93
:101E00001CAA1FAA1EAA19AE18AEBE01665C7F4F9F
:101E1000CE01C4960E944906BE01625D7F4FCE018D
:101E2000C4960E94C605B8010E94C60522961FAE40
:101E30001EAE229724961FAE1EAE249726961FAE86
:101E40001EAE2697BC01CE01805C9F4F0E944906C2
:101E5000CE01C4960E949605CE01CA960E949605B0
:101E6000CE018E960E949605C8010E949605CE016D
:101E7000805C9F4F0E94400597FD21C06F3F710518
:101E80008105910509F0F4F4F601619371936F01F6
:101E9000CE01805C9F4F0E949605F3E0EF0EF11C8F
:101EA00021E1E216F10409F062CF53CFEE0DFF1DE0
:101EB00070CFE80FF91F85CFE80FF91F9BCF70E0B7
:101EC00060E0E2CF6FEF70E0DFCFCE018A5B9F4F23
:101ED0000E944005672B39F41092970160E082E080
:101EE0000E94BA0136CF81E08093970161E0F7CF7D
:101EF000CE018A5B9F4F0E9440054B011092AC01BE
:101F00001092AB0181E090E09093A4018093A30133
:101F100010929201109291010E94EE048CE3889D30
:101F20007001899DF00C1124C7010E94A6038091C5
:101F3000A7019091A801E80EF91EF092A801E09285
:101F4000A7010E94BE041092A4011092A30182E096
:101F500090E09093A6018093A5010E94EE048091E9
:101F6000AA018F938091A9018F938091A8018F93EB
:101F70008091A7018F939F928F928BE591E09F9321
:101F80008F931F930F930E946816B8018DE44FCE74
:101F900080911703843450F1809153029091540240
:101FA000825491098E9710F590E080E040E050E077
:101FB000BA01FC01EB5AFD4F2081318129503109D2
:101FC0002930310598F4FC01E95AFD4F2081318117
:101FD000265131092131310508F488C02081318131
:101FE000265031092730310508F499C096E02916AA
:101FF00031040CF414CDAAE4B2E06496BFAFAEAFE6
:102000006497E3E0F0E06696FFAFEEAF669795EC7D
:10201000C92E9DE9D92E9CE1E92E91E8F92E66960C
:102020008EAD9FAD6697821593050CF07DC06496CA
:10203000AEADBFAD64971B966D917C911C971796C2
:10204000AD90BC9090E080E00E9441122B013C01D9
:10205000B50190E080E00E9441124B015C012DEC43
:102060003CEC4CE45FE30E94A2129B01AC01C30173
:10207000B2010E943C12F0E0E0E087FD14C02DECBC
:102080003CEC4CE45FE3C301B2010E94A2129B014D
:10209000AC01C501B4010E943C12E2E0F0E087FD12
:1020A00002C0E1E0F0E0A701960163E971E080E0A1
:1020B00091E00E94C7136F01FF0FEE08FF08C626CC
:1020C000D726E826F9266696EEADFFAD66973196DF
:1020D0006696FFAFEEAF669764968EAD9FAD649740
:1020E000029664969FAF8EAF649799CF440F551FA9
:1020F000661F771F416004968038910509F059CF1B
:1021000080E290E09093880180938701409383015F
:102110005093840160938501709386011CCC440F19
:10212000551F661F771FE7CFC0928301D0928401AD
:10213000E0928501F092860180E290E09093880120
:10214000809387018FEF9FEF08CC80937B01909362
:102150007C01A0937D01B0937E0120919301309189
:1021600094012130310509F01BCC8D33F2EC9F072F
:10217000FAE9AF07F6EABF0731F087369849AA496E
:10218000B64A09F00DCC4091A20164E670E081E00E
:1021900090E00E947E0404CC8735F8EA9F07FAE9B4
:1021A000AF07F6EABF0709F492C08D3322EC92071D
:1021B0002AE9A20726EAB20709F4E2C08D35924A5D
:1021C000AA49B64A09F00ECC4091A20164E670E03B
:1021D00081E090E00E947E048091AB019091AC017F
:1021E0008130910591F4209191013091920121303B
:1021F000310509F09BC01092A6011092A5018091B3
:10220000A9019091AA010E94F4044091A20164E600
:1022100070E082E090E00E947E04E4CB4091A20155
:1022200064E670E081E090E00E947E04809193017A
:1022300090919401009789F481E090E0909394014B
:10224000809393018FEF9FEF90937A0180937901B0
:10225000809195019091960108C0019741F41092E8
:1022600094011092930190E080E00E9429030E9463
:10227000EE04B8CB8091930190919401019709F0FD
:10228000B1CB4091A20164E670E081E090E00E9451
:102290007E048091790190917A018430910514F047
:1022A00083E090E07C01FFEFEF1AFF0AF0927A01E1
:1022B000E092790124E0E216F10461F54091A20177
:1022C00064E670E082E090E00E947E0423C080918A
:1022D000930190919401019709F084CB4091A20160
:1022E00064E670E081E090E00E947E0480917901D4
:1022F00090917A011816190614F081E090E07C01A3
:10230000A1E0EA1AF108F0927A01E0927901E11471
:10231000F104A1F2F701EE0FFF1FE357FE4F838593
:10232000948590939601809395019FCF223031053B
:1023300009F06BCF9093A6018093A5018091A9012C
:102340009091AA019195819591095DCF209193017A
:10235000309194012130310509F044CB80919501F1
:10236000909196010197181619062CF490939601F6
:10237000809395016DCF309396012093950168CF9E
:102380008091930190919401019709F02BCB80915A
:1023900095019091960101968F3F91053CF3EFEFE7
:1023A000F0E0F0939601E093950152CFCF93DF9345
:1023B000C0911E03D0911F032097E1F0FE013297D8
:1023C0002081318146E0429FC001439F900D11243E
:1023D000C80FD91F9E0180911E0390911F0326975D
:1023E0008217930721F0CE010E949605F3CF029742
:1023F0000E94E21482E293E0DF91CF910C94960563
:102400001F93FC0199278827BC01E8941191103291
:10241000E9F3193010F01E30C8F31B3251F01D32B1
:1024200049F4689406C00E942712610F711D811D36
:10243000911D119110531A30B0F33EF49095809590
:10244000709561957F4F8F4F9F4F1F910895592F22
:10245000482F372F262F660F771F881F991F660F6B
:10246000771F881F991F620F731F841F951F660FA8
:10247000771F881F991F08950E947E1208F481E03B
:102480000895E89409C097FB3EF490958095709567
:1024900061957F4F8F4F9F4F9923A9F0F92F96E9B0
:1024A000BB279395F695879577956795B795F11125
:1024B000F8CFFAF4BB0F11F460FF1BC06F5F7F4FC2
:1024C0008F4F9F4F16C0882311F096E911C07723D4
:1024D00021F09EE8872F762F05C0662371F096E8DD
:1024E000862F70E060E02AF09A95660F771F881FAC
:1024F000DAF7880F9695879597F90895990F000850
:10250000550FAA0BE0E8FEEF16161706E807F907C5
:10251000C0F012161306E407F50798F0621B730B60
:10252000840B950B39F40A2661F0232B242B252BE1
:1025300021F408950A2609F4A140A6958FEF811D84
:10254000811D08950E94B5120C9426130E94181341
:1025500038F00E941F1320F0952311F00C940F13F4
:102560000C94151311240C945A130E94371370F312
:10257000959FC1F3950F50E0551F629FF001729F28
:10258000BB27F00DB11D639FAA27F00DB11DAA1F37
:10259000649F6627B00DA11D661F829F2227B00D84
:1025A000A11D621F739FB00DA11D621F839FA00D0F
:1025B000611D221F749F3327A00D611D231F849F5F
:1025C000600D211D822F762F6A2F11249F575040B6
:1025D0009AF0F1F088234AF0EE0FFF1FBB1F661F31
:1025E000771F881F91505040A9F79E3F510580F0FA
:1025F0000C940F130C945A135F3FE4F3983ED4F3FA
:10260000869577956795B795F795E7959F5FC1F79D
:10261000FE2B880F911D9695879597F9089597F948
:102620009F6780E870E060E008959FEF80EC089578
:1026300000240A94161617061806090608950024A1
:102640000A9412161306140605060895092E03941B
:10265000000C11F4882352F0BB0F40F4BF2B11F48F
:1026600060FF04C06F5F7F4F8F4F9F4F089557FDEE
:102670009058440F551F59F05F3F71F04795880FF0
:1026800097FB991F61F09F3F79F087950895121687
:1026900013061406551FF2CF4695F1DF08C0161633
:1026A00017061806991FF1CF8695710561050894E4
:1026B0000895E894BB2766277727CB0197F90895FB
:1026C000F999FECF92BD81BDF89A992780B50895FA
:1026D000262FF999FECF1FBA92BD81BD20BD0FB63E
:1026E000F894FA9AF99A0FBE019608950E94B813C9
:1026F000A59F900DB49F900DA49F800D911D112456
:1027000008952F923F924F925F926F927F928F9295
:102710009F92AF92BF92CF92DF92EF92FF920F9370
:102720001F93CF93DF93CDB7DEB7CA1BDB0B0FB67A
:10273000F894DEBF0FBECDBF09942A883988488837
:102740005F846E847D848C849B84AA84B984C884CD
:10275000DF80EE80FD800C811B81AA81B981CE0FC4
:10276000D11D0FB6F894DEBF0FBECDBFED010895A9
:10277000A29FB001B39FC001A39F700D811D1124C2
:10278000911DB29F700D811D1124911D0895DB01D3
:102790008F939F930E947613BF91AF91A29F800D5C
:1027A000911DA39F900DB29F900D1124089597FB4A
:1027B000072E16F4009407D077FD09D00E9410145C
:1027C00007FC05D03EF4909581959F4F0895709534
:1027D00061957F4F0895052E97FB1EF400940E948B
:1027E000021457FD07D00E94241407FC03D04EF4B6
:1027F0000C94021450954095309521953F4F4F4FC2
:102800005F4F089590958095709561957F4F8F4F9C
:102810009F4F0895EE0FFF1F0590F491E02D09944E
:10282000AA1BBB1B51E107C0AA1FBB1FA617B707F6
:1028300010F0A61BB70B881F991F5A95A9F7809512
:102840009095BC01CD010895A1E21A2EAA1BBB1BD5
:10285000FD010DC0AA1FBB1FEE1FFF1FA217B3076C
:10286000E407F50720F0A21BB30BE40BF50B661F82
:10287000771F881F991F1A9469F760957095809546
:1028800090959B01AC01BD01CF0108950F931F935B
:10289000CF93DF938230910510F482E090E0E091D5
:1028A0004403F091450330E020E0B0E0A0E0309731
:1028B00099F42115310509F44AC0281B390B24303D
:1028C0003105D8F58A819B816115710589F1FB017C
:1028D00093838283FE0111C0408151810281138163
:1028E00048175907E0F04817590799F4109761F015
:1028F00012960C93129713961C933296CF01DF9188
:10290000CF911F910F9108950093440310934503B5
:10291000F4CF2115310551F04217530738F0A901C2
:10292000DB019A01BD01DF01F801C1CFEF01F9CF51
:102930009093450380934403CDCFFE01E20FF31F34
:10294000819391932250310939832883D7CF2091E5
:10295000420330914303232B41F420910201309133
:1029600003013093430320934203209100013091EF
:1029700001012115310541F42DB73EB74091040105
:1029800050910501241B350BE0914203F091430364
:10299000E217F307A0F42E1B3F0B2817390778F036
:1029A000AC014E5F5F4F2417350748F04E0F5F1F95
:1029B0005093430340934203819391939FCFF0E060
:1029C000E0E09CCFCF93DF930097E9F0FC013297D2
:1029D00013821282A0914403B0914503ED0130E0CF
:1029E00020E01097A1F420813181820F931F209164
:1029F0004203309143032817390709F061C0F0936F
:102A00004303E0934203DF91CF910895EA01CE178B
:102A1000DF07E8F54A815B819E0141155105B1F759
:102A2000E901FB83EA8349915991C40FD51FEC1743
:102A3000FD0761F4808191810296840F951FE90161
:102A400099838883828193819B838A83F0E0E0E08D
:102A500012968D919C9113970097B9F52D913C9109
:102A60001197CD010296820F931F2091420330915E
:102A700043032817390739F6309751F5109245036B
:102A800010924403B0934303A0934203BCCFD3837B
:102A9000C28340815181840F951FC817D90761F403
:102AA0004E5F5F4F88819981480F591F5183408342
:102AB0008A819B81938382832115310509F0B0CFF0
:102AC000F0934503E09344039ECFFD01DC01C0CFAA
:102AD00013821282D7CFB0E0A0E0E1E7F5E10C94D9
:102AE00083138C01009751F4CB010E9446148C0192
:102AF000C801CDB7DEB7E0E10C949F13FC01E60FEF
:102B0000F71F9C0122503109E217F30708F49DC01A
:102B1000D901CD91DC911197C617D70798F0C53030
:102B2000D10530F3CE0104978617970708F3C61B2B
:102B3000D70B2297C193D1936D937C93CF010E94C1
:102B4000E214D6CF5B01AC1ABD0A4C018C0E9D1E5F
:102B5000A0914403B0914503512C412CF12CE12C60
:102B6000109731F5809142039091430388159905A0
:102B700009F05CC04616570608F058C08091000165
:102B800090910101009741F48DB79EB740910401E7
:102B900050910501841B950BE817F90708F055C003
:102BA000F0934303E0934203F90171836083A0CF64
:102BB0008D919C91119712966C90129713967C9020
:102BC0001397A815B90559F56C0142E0C40ED11C44
:102BD000CA14DB0420F1AC014A195B09DA01129630
:102BE000159780F06282738251834083D9016D937F
:102BF0007C93E114F10471F0D7011396FC93EE93EA
:102C0000129776CF22968C0F9D1FF90191838083B6
:102C1000F301EFCFF0934503E093440369CF4816E7
:102C2000590608F42C017D01D3019ACFCB010E94F3
:102C300046147C01009749F0AE01B8010E942816A5
:102C4000C8010E94E214870153CF10E000E050CF8A
:102C5000FB01DC0102C001900D9241505040D8F7B9
:102C60000895FB01DC0101900D920020E1F7089529
:102C7000AEE0B0E0EEE3F6E10C948F130D891E890F
:102C80008F89988D26E02C831A83098397FF02C0D1
:102C900080E090E801979E838D83AE01455E5F4F93
:102CA000698D7A8DCE0101960E948B164D815E81D1
:102CB00057FD0AC02F813885421753070CF49A013B
:102CC000020F131FF80110822E96E4E00C94AB1350
:102CD000AEE0B0E0EEE6F6E10C948F130D891E89AC
:102CE00086E08C831A8309838FEF9FE79E838D8311
:102CF000AE01475E5F4F6F89788DCE0101960E94CD
:102D00008B162F813885020F131FF80110822E9623
:102D1000E4E00C94AB13ABE0B0E0E1E9F6E10C9435
:102D200081137C013B018A01FC0117821682838199
:102D300081FFC8C1CE0101965C01F7019381F301C7
:102D400093FD859193FF81913F01882309F453C13D
:102D5000853239F493FD859193FF81913F0185324E
:102D600029F4B70190E00E947B18E7CF912C212C29
:102D7000312CFFE1F31538F08B3211F190F48032F1
:102D800009F1833229F137FC3CC020ED280F2A30AD
:102D900050F536FE20C08AE0989E200D1124922E18
:102DA00006C08D3291F0803371F7689430F8F301EA
:102DB00093FD859193FF81913F018111DACF21C06D
:102DC000689431F8689432F8F2CF689433F8EFCF12
:102DD000689434F8ECCFEAE02E9E200D1124222EC8
:102DE000689435F8E4CF8E3229F436FC04C1689437
:102DF00036F8DDCF8C3619F4689437F8D8CF88369A
:102E0000B1F2982F9F7D95549330E0F08336A1F175
:102E10008337C1F1833509F063C02801F2E04F0E1A
:102E2000511CF801C080D180692D70E036FC02C0D1
:102E30006FEF7FEFC6010E9465184C01689437F868
:102E400082010AC00C5F1F4FFFE3F983882483943B
:102E5000912C6501E89437F833FE2DC0522C811473
:102E6000910471F5552009F468CFB70180E290E034
:102E70000E947B185A94F6CFF801808189830E5FF7
:102E80001F4FE4CF2801F2E04F0E511CF801C08023
:102E9000D180692D70E036FC02C06FEF7FEFC60174
:102EA0000E9470184C018201D5CFB70180E290E0FA
:102EB0000E947B182A942814190409F0B0F7CECF89
:102EC000F60137FC859137FE81916F01B70190E0E3
:102ED0000E947B1851105A94F1E08F1A9108BFCFCD
:102EE000843619F0893609F077C0F80137FE6BC0D7
:102EF00060817181828193810C5F1F4FF32DFF767A
:102F00003F2E97FF09C090958095709561957F4FF2
:102F10008F4F9F4F689437F82AE030E0A5010E9458
:102F2000AB18C82ECA188C2C432C36FE0CC0E89463
:102F300040F8C91440F434FE05C032FC03C0F32D40
:102F4000FE7E4F2E892C44FE95C0FE01EC0DF11D36
:102F50008081803309F087C0242D297E422E842D64
:102F60008870582E43FC95C040FE8FC09C2C821464
:102F700018F42C0C922C981844FE91C0B70180E3F1
:102F800090E00E947B1842FE09C088E790E041FE75
:102F900002C088E590E0B7010E947B18C91408F4CC
:102FA0008AC0CA94D12C9FEFC91AD90ACA0CDB1C5B
:102FB000F60182916F01B70190E00E947B18AC147A
:102FC000BD04B1F74FCF60817181072E000C880BD3
:102FD000990B0E5F1F4F92CFD32CE894D4F82AE0C0
:102FE00030E0853739F1232D297FD22E8F3601F13C
:102FF00048F48835A9F0F701868197812B96E2E1A4
:103000000C949D13803749F08837A9F7D4FE02C08D
:103010006894D2F820E130E00DC06894D4F8F6CF7F
:1030200034FE03C0822F8660D82E20E132E002C039
:1030300028E030E0F801D7FE0FC060817181828105
:1030400093810C5F1F4FA5010E94AB18C82ECA18B0
:103050003D2CE89437F867CF6081718190E080E083
:103060000E5F1F4FF0CF42FC02C0839478CF839451
:10307000839475CF842D867809F471CFF6CFB7018C
:1030800080E290E00E947B1883948214C0F3512C5C
:1030900073CF522C5818821408F46ECFF8CF842DB9
:1030A000867809F47BCF8BE241FE80E247FC8DE21B
:1030B000B70190E071CFB70180E390E00E947B18E8
:1030C0009A946CCF8FEF9FEF99CFFC0105906150E0
:1030D00070400110D8F7809590958E0F9F1F08952E
:1030E000FC016150704001900110D8F780959095D7
:1030F0008E0F9F1F08950F931F93CF93DF93182F69
:10310000092FEB018B8181FD09C01FEF0FEF812F8C
:10311000902FDF91CF911F910F91089582FF14C0DE
:103120002E813F818C819D81281739073CF4E881ED
:10313000F981CF0101969983888310838E819F81C5
:1031400001969F838E83E3CFE885F985812F0995CA
:10315000892BA1F3DACFFA01AA27283051F12031C7
:1031600081F1E8946F936E7F6E5F7F4F8F4F9F4F1B
:10317000AF4FB1E03ED0B4E03CD0670F781F891F5D
:103180009A1FA11D680F791F8A1F911DA11D6A0F2B
:10319000711D811D911DA11D20D009F468943F91DE
:1031A0002AE0269F11243019305D3193DEF6CF01DD
:1031B0000895462F4770405D4193B3E00FD0C9F7A3
:1031C000F6CF462F4F70405D4A3318F0495D31FD10
:1031D0004052419302D0A9F7EACFB4E0A695979563
:1031E000879577956795BA95C9F700976105710539
:1031F00008959B01AC010A2E069457954795379583
:103200002795BA95C9F7620F731F841F951FA01DDC
:10321000089510E0C2E6D0E004C0FE010E940A1446
:0C3220002196C336D107C9F7F894FFCF00
:10322C000000460380003430350047656D696E69D7
:10323C00466C617450616E656C00000000002401E6
:10324C008E00BB007101EC00CA00DE002A2563254C
:10325C00732563002A256325642563004F70656E12
:10326C00656400436C6F7365640025642564256494
:10327C0025640025645265616479005374256443A8
:08328C006125644F6125640017
:00000001FF
